:020000008E2848
:10000800F000030E8312F1000928710E8300F00E30
:10001800700E0900230882071428152817281A28A3
:1000280008000000080000000000080000000000B0
:10003800000008000301A200051820282408A300D6
:10004800A30B2428A20F29280800051C2228080031
:100058000301A200051C2E282408A300A30B3228A4
:10006800A20F372808000518302808002708A20022
:1000780085140E2000000000000085100E200000EE
:100088000000000085140E2000000000000085100C
:100098000E20A20B3C282808A20085100E20000084
:1000A8000000000085100E200000000000008510F0
:1000B8000E2000000000000085100E20A20B512821
:1000C80008002508A0002B08A20026187028A10DFA
:1000D800031C70282C08A2008514000000000000F2
:1000E8000E2085100E20A20B70282D08A200261CB9
:1000F8008228A10D031C82282E08A200851000006A
:10010800000000000E2085100E20A20B8228A00BF4
:100118006728080007309F00831685100514061409
:100128008312851035224C2207398207A228CD2850
:100138003B297729072A152A972897284C22B300A4
:100148004C22B4004C22B5004C22B6000830A50061
:100158000130A600AD30A7005630A8001530AB001E
:100168001530AC001530AD004030AE003A203308F1
:10017800A10065203408A10065203508A10065208C
:100188003608A10065201530A7007030A8003A2075
:1001980097284C22A3004C22AB004C22AD004C22E5
:1001A800AC004C22AE004C22A7004C22A8004C22E6
:1001B800A9004C22AA004C22B0004C22B1004C22CB
:1001C800B2004C22B3004C22B9004C22B4004C229D
:1001D800BA004C22B5004C22BB004C22B6004C227F
:1001E800BC004C22B7004C22BD004C22B8004C2267
:1001F800BE000830A5000130A6003A203008A10052
:1002080065203108A10065203208A1006520390861
:1002180003191229A5003308A10065203A0803191B
:100228001929A5003408A10065203B0803192029D5
:10023800A5003508A10065203C0803192729A50059
:100248003608A10065203D0803192E29A5003708A6
:10025800A10065203E0803193529A5003808A1002A
:1002680065202908A7002A08A8003A209728051819
:100278003B291F30A4002C2022081E3C03183F29CC
:100288001F30A4000830A0002C2022080A3CB30D1F
:10029800A00B48290830A0002C2022080A3CB40DE5
:1002A800A00B50290830A0002C2022080A3CB50DCC
:1002B800A00B58290830A0002C2022080A3CB60DB3
:1002C800A00B6029FF30B306FF30B406FF30B50637
:1002D800FF30B6063308462234084622350846223F
:1002E8003608462297284C22B9004C22BA004C22E4
:1002F800BB004C22BC004C22BD004C22BE00B30106
:10030800B401B501B601B701B801051889291F3034
:10031800A4002C2022080E3C03188D291F30A400AD
:100328000830A0002C2022080A3CB00DA00B96290A
:100338000830A0002C2022080A3CB10DA00B9E29F1
:100348000830A0002C2022080A3CB20DA00BA629D8
:1003580039080319B5292C2022080A3CB30DB90B1A
:10036800AF293A080319BE292C2022080A3CB40DEB
:10037800BA0BB8293B080319C7292C2022080A3CC4
:10038800B50DBB0BC1293C080319D0292C20220824
:100398000A3CB60DBC0BCA293D080319D9292C20E3
:1003A80022080A3CB70DBD0BD3293E080319E229E0
:1003B8002C2022080A3CB80DBE0BDC29FF30B00601
:1003C800FF30B106FF30B206FF30B306FF30B40687
:1003D800FF30B506FF30B606FF30B706FF30B80667
:1003E800300846223108462232084622330846227F
:1003F800340846223508462236084622370846225F
:100408003808462297282F30A4000301A000A00A2C
:100418001E202C2003012202031D0B2A200846223D
:1004280097281F30A4004C22A000A1008313A030FD
:1004380084001E2022088000840A2C2022088000C4
:10044800840AA10B1D2A2008A1008313A030840070
:1004580000084622840A00084622840AA10B2C2A96
:1004680097281A30831699001815181283129817AE
:1004780083160C12181398168C12831218139811DD
:100488001816080099008316981C482A8312080039
:100498008C1E4C2A1A081819542A9818542A08002D
:0604A800981598110800F0
:02400E00183F59
:00000001FF
